Share this
Analyzing SQL Server Data File Anatomy
by Murilo Miranda on Nov 2, 2012 12:00:00 AM
A database is a defined space stored in the system, grouping user objects. This space can be split into several files organized in groups.
In SQL Server, you have a limit of 32,767 databases per instance, and each database can store more than 2 billion objects, reaching a physical size up to 524,272 terabytes!!!
In this post, I will explain the physical structure of a SQL Server data file in greater depth. Unfortunately, I cannot write all the assumptions, behaviors, and details on this topic, but you will read a good overview of a file structure and a good starting point to better understand index internals, file fragmentation, transaction log internals, and so on…
Before we start, let’s remember some vital concepts.
Database Files
You can see a database file as a normal operating system file. A database must have a least two files: one for data and one for t-logs.
The data files are categorized into two types: Master Data File and Secondary Data File(s). Only one Master Data File is possible for each database, and it keeps track of all the other files in the database. By convention, the Master Data File has the .mdf extension and the secondary files have .ndf.
For the log files, the extension is .ldf. Each database must have at least one.
Page Structure
In Microsoft, the fundamental unit of data storage in SQL Server is the page. The disk space allocated to a data file (.mdf or .ndf) in a database is logically divided into pages numbered contiguously from 0 to n. Disk I/O operations are performed at the page level. That is, SQL Server reads or writes whole data pages.
All the pages in SQL Server have the same structure. At the top of the page there’s a 96 bytes header, and it includes the PageID, the kind of structure the page belongs to, the number of records in the page, and pointers to the previous and next pages. So there are 8096 bytes available on which we can store records. However, the maximum length of data records is 8060 bytes, as in the bottom of the page (latest 36 bytes), resides the slot array containing information about the offset of the rows (2 bytes per row). This array can grow from bottom to top based on the size of the records, so more records can be accommodated in a page and offset table will take more space. These slots are stored in the order defined by index key. For heaps, there’s no special order.
Space Allocation
The space allocation in SQL Server is managed in portions called “extents”, which are basically a group of eight logically contiguous pages. So, a lot of 64 KB (8*8 KB/Page).
The use of extents makes the allocation system more efficient. These units can be distinguished in two types:
- Uniform extents: Extent units composed by pages owned by a single object
- Mixed extents: Extent units composed by pages shared to up to eight objects.
The pages are allocated for a new table or index starting from a mixed extent. When the object grows to eight pages, all future allocations will use uniform extents.
All the information about the extents is tracked in GAM, SGAM, and IAM pages, also known as “allocation bitmaps”.
File Structure
Basically, a SQL Server data file has the following basic structure, which we will analyze:
- Page 0: Header
- Page 1: First PFS
- Page 2: First GAM
- Page 3: First SGAM
- Page 4: Unused
- Page 5: Unused
- Page 6: First DCM
- Page 7: First BCM
File Header
All the files have a header into the page number 0. This header stores metadata about that particular file and is not recoverable by checkdb. In case of damage, you must restore the entire file.
You can explore the header of some database using the following DBCC command:
DBCC fileheader [( {‘dbname’ | dbid} [, fileid])
You will find useful information on RedoStartLSN, BindingId, SectorSize, Status, and Growth records.
Page Free Space
The PFS identifies the allocation status and determines the amount of free space. These pages contain 1 byte for each page and cover a range of 8,088 pages in a file.
The basic PFS structure is:
- Bit 1: Indicates whether the page is allocated or not.
- Bit 2: Indicates if the page is from a mixed extent.
- Bit 3: Indicates that this page is an IAM page.
- Bit 4: Indicates that this page contains ghost records
- Bits 5 to 7: A combined three-bit value, which indicate the page fullness as follows:
- 0: The page is empty
- 1: The page is 1–50% full
- 2: The page is 51–80% full
- 3: The page is 81–95% full
- 4: The page is 96–100% full
The first page of each file is a PFS, and another PFS is allocated for every 8,000 pages after the first PFS.
After an extent has been allocated to an object, the Database Engine uses the PFS pages to record which pages in the extent are allocated or free. The SQL Server allocates a new extent only when it cannot find a page with sufficient space to hold the data.
GAM and SGAM
SQL Server uses two special types of pages to record which extents have been allocated and for which type of use (mixed or uniform) the extent is available:
Global Allocation Map (GAM) pages: Tracks the allocation of any type of extents. A GAM has a bit for each extent in the interval this covers. The bit 0 means that the corresponding extent is in use, and in other hands, the bit is 1 tracks free extents. A GAM can cover about 64,000 extents, or almost 4 GB of data. So, there is one GAM page for every 4 GB of file size.
Shared Global Allocation Map (SGAM) pages: This is the same as GAM, but it refers only to mixed extents. The SGAM has a bit for each extent in the interval it covers. If the bit is 1, the used extent is a mixed extent and has free pages, and the 0 bit represents either a non-mixed extent or a mixed extent whose pages are all in use.
Differential Changed Map (DCM)
It is the seventh page (page 6). It keeps track of which extents in a file have been modified since the last full database backup.
Like GAM and SGAM, BCM pages have 1 bit for each extent in its covered sector of the file. The first BCM page is on the seventh page of every data file and at every 511,230 pages thereafter.
Bulk Changed Map (BCM)
Also known as Minimally Logged Map (ML Map), it is the eighth page (page 7) and is used when an extent in the file is used in a minimally or bulk-logged operation.
Each bit on a BCM page represents an extent, and if the bit is 1, this extent has been changed by a minimally-logged bulk operation since the last transaction log backup. The first BCM page is on the eighth page of every data file and at every 511,230 pages thereafter. All the bits on a BCM page are reset to 0 every time a log backup occurs.
The Boot Page
The page 9 in file 1 is perhaps the most important page in the database – the Boot Page. The base metadata about the whole database is stored in this page. If this page is corrupt, checkdb cannot repair this page, and a restore of file number 1 will be needed to recover the database.
To get information about the database boot page, you can execute DBCC PAGE pointing to page 9 in file 1 or DBCC dbinfo [(‘dbname’)], always activating the trace flag 3604 (DBCC TRACEON(3604)).
Index Allocation Map – IAM Pages
The function of IAM pages is to track the extents that belong to tables or indexes. The IAM is a bitmap that refers extents to objects. This kind of page covers a 4-GB range, belongs to a GAM interval, and is not located at known locations in a file.
For each 4-GB range of data, partition, and allocation unit type, an IAM page is required to track.
By the way, an Allocation Unit is a group of pages that manage data based on their page type and can be from three types:
- IN_ROW_DATA: Data or index rows that contain all data, except large object (LOB) data.
- LOB_DATA: Large object data stored in one or more of these data types: text, ntext, image, xml, varchar(max), nvarchar(max), varbinary(max), or CLR user-defined types.
- ROW_OVERFLOW_DATA: Variable length data stored in varchar, nvarchar, varbinary, or sql_variant columns that exceed the 8,060 byte row size limit.
For example, a table on four partitions that has all three types of data (in-row, LOB, and row-overflow) has at least 12 IAM pages.
There are four possible combinations of the above pages that are valid for an extent:
IAM Chains
Knowing that a single IAM page covers a 4-GB range (512.000 pages) in a file and belongs to a single GAM interval, what happens if the allocation unit contains extents from more than one file or more than one 4-GB range of a file? There will be multiple IAM pages linked in an IAM chain, an unordered sequence of IAM pages.
Basically, an IAM page has a header containing information about which GAM interval this belongs to, the sequence number, and the linkage information.
Demo
For these demos, I will use the AdventureWorks2008R2 database to make a simpler reproduction. You can download this sample database, and others, on https://msftdbprodsamples.codeplex.com/.
Demo 1: Page Anatomy and PFS, GAM, SGAM, DCM and BCM demonstration
So let’s start demonstrating the Allocation Bitmaps. The %%lockres%% and %%physloc%% mechanisms will return the physical location of the row. So I’m going to use the following query to return the first 5 rows of databaselog table, showing the physical location of each row.
SELECT TOP(5) a .%% physloc %% as Address,
a .%% lockres %% as LockHashValue,
a.*
FROM dbo.databaselog AS a
I got the following rows, and I will explore the second row.
To explore the second row internals, I will use the Database Console Command (DBCC) PAGE for it. Notice that 1:150:1 represents FILE:PAGE:SLOT. So here is the command, using page 150:
DBCC traceon(3604) — We need to activate this flag before execute the DBCC PAGE
DBCC page (adventureworks2008r2, 1, 150, 2)
DBCC traceoff(3604)
The execution returned a long result, but for now let’s concentrate on Allocation Status in the Header section:
Allocation Status
GAM (1:2) = ALLOCATED SGAM (1:3) = NOT ALLOCATED
PFS (1:1) = 0x63 MIXED_EXT ALLOCATED 95_PCT_FULL DIFF (1:6) = CHANGED
ML (1:7) = NOT MIN_LOGGED
Basically we can get all the allocation information about this page and the PFS, GAM, SGAM, DCM, and BCM, which is tracking this page.
After the page Header, we have the data. Here is a sample:
lot 0, Offset 0x60, Length 2732, DumpStyle BYTE
Record Type = PRIMARY_RECORD Record Attributes = NULL_BITMAP VARIABLE_COLUMNS
Record Size = 2732
Memory Dump @0x0000000009ABA060
0000000000000000: 30001000 01000000 5d85e400 23a00000 †0…….]ä.# ..
0000000000000010: 08000006 0027003f 00450055 00db03ac †…..’.?.E.U.Û.¬
0000000000000020: 0a640062 006f0043 00520045 00410054 †.d.b.o.C.R.E.A.T
0000000000000030: 0045005f 00540041 0042004c 00450064 †.E._.T.A.B.L.E.d
0000000000000040: 0062006f 00450072 0072006f 0072004c †.b.o.E.r.r.o.r.L
0000000000000050: 006f0067 00430052 00450041 00540045 †.o.g.C.R.E.A.T.E
0000000000000060: 00200054 00410042 004c0045 0020005b †. .T.A.B.L.E. .[
0000000000000070: 00640062 006f005d 002e005b 00450072 †.d.b.o.]…[.E.r
0000000000000080: 0072006f 0072004c 006f0067 005d0028 †.r.o.r.L.o.g.].(
0000000000000090: 000d000a 00200020 00200020 005b0045 †….. . . . .[.E
00000000000000A0: 00720072 006f0072 004c006f 00670049 †.r.r.o.r.L.o.g.I
And to conclude, the row offset. This way, you can see all the three parts of the page anatomy, as explained earlier in this article:
OFFSET TABLE:
Row – Offset
5 (0x5) – 7017 (0x1b69)
4 (0x4) – 6774 (0x1a76)
3 (0x3) – 5713 (0x1651)
2 (0x2) – 4560 (0x11d0)
1 (0x1) – 2828 (0xb0c)
0 (0x0) – 96 (0x60)
Demo 2: Looking to IAM
Now I will execute a query that will return all allocation units for the table DatabaseLog. For this I will relate sys.partitions and sys.system_internals_allocation_units DMV, and for each allocation unit we can get the page info, which guides us to the IAM info/chain.
I’m using a page conversion algorithm done by Kimberley Tripp (https://sqlskills.com/blogs/paul/post/Inside-The-Storage-Engine-sp_AllocationMetadata-putting-undocumented-system-catalog-views-to-work.aspx).
So, here’s the query:
SELECT Object_name(p.object_id) AS ‘tableName’,
i.name AS ‘indexName’,
p.partition_number,
au.type_desc,
CONVERT (VARCHAR(6), CONVERT (INT, Substring (au.first_page, 6, 1) +
Substring (
au.first_page, 5, 1)))
+ ‘:’
+ CONVERT (VARCHAR(20), CONVERT (INT, Substring (au.first_page, 4, 1) +
Substring (au.first_page, 3, 1) + Substring (au.first_page, 2, 1) +
Substring (
au.first_page, 1, 1))) AS ‘firstPage’,
CONVERT (VARCHAR(6), CONVERT (INT, Substring (au.root_page, 6, 1) +
Substring (
au.root_page, 5, 1)))
+ ‘:’
+ CONVERT (VARCHAR(20), CONVERT (INT, Substring (au.root_page, 4, 1) +
Substring
(au.root_page, 3, 1) + Substring (au.root_page, 2, 1) + Substring
(au.root_page,
1, 1))) AS ‘rootPage’,
CONVERT (VARCHAR(6), CONVERT (INT, Substring (au.first_iam_page, 6, 1) +
Substring (au.first_iam_page, 5, 1)))
+ ‘:’
+ CONVERT (VARCHAR(20), CONVERT (INT, Substring (au.first_iam_page, 4, 1)
+
Substring (au.first_iam_page, 3, 1) + Substring (au.first_iam_page, 2, 1)
+
Substring (au.first_iam_page, 1, 1))) AS ‘firstIamPage’
FROM sys.indexes AS i
JOIN sys.partitions AS p
ON i.object_id = p.object_id
AND i.index_id = p.index_id
JOIN sys.system_internals_allocation_units AS au
ON p.hobt_id = au.container_id
WHERE p.object_id = Object_id(‘databaselog’)
ORDER BY tablename;
And here is the result (Notice that when executing the DBCC IND, you can have the same info in a more fragmented layout):
If we execute the DBCC PAGE into the root page in option 3, we can get all the IAM chain belonging to the allocation unit. In this case, I choose the IN_ROW_DATA belonging to the clustered index PK_DatabaseLog_DatabaseLogID.
DBCC traceon(3604)
DBCC page (adventureworks2008r2, 1, 1270, 3)
DBCC traceoff(3604)
In the output, checking the ChildPageID, it’s possible to observe all the pages owned by the chain, in the proper sequence:
So now you can explore all the data belonging to this allocation unit using the DBCC PAGE. In this IAM demo, it was possible to verify all the allocation units of the referred table, in this case four, and check the IAM Chain of one of those allocation units.
Demo 3: We know about tables now, but… Where are the other objects?
Where are the Stored Procedures, Views, functions? Obviously, stored into the same file structure! But…how do we reach this?
To demonstrate this, we will need to connect using the Dedicated Administrator Connection (DAC) in order to access sys.sysobjvalues. In this case, I’m crossing sys.sysobjvalues with sysobjects table and just showing the objects with type “P” (Stored Procedures). Here is the query:
SELECT v .%% physloc %% as address,
CONVERT (VARCHAR(6), CONVERT (INT, Substring (v.%%physloc%%, 6, 1) +
Substring (
v.%%physloc%%, 5, 1)))
+ ‘:’
+ CONVERT (VARCHAR(20), CONVERT (INT, Substring (v.%%physloc%%, 4, 1) +
Substring (v.%%physloc%%, 3, 1) + Substring (v.%%physloc%%, 2, 1) +
Substring (v
.%%physloc%%, 1, 1))) AS ‘rootPage’,
o.name objectName,
Cast(v.imageval AS VARCHAR(max)) code
FROM sys.objects o
INNER JOIN sys.sysobjvalues v
ON o.object_id = v.objid
WHERE o.type = ‘P’
Here is the output:
Voilà! Now you know the exact page on which your object is stored, and you can explore it. It’s also possible to decrypt the code, if the procedure is encrypted. I recommend reading this article: https://williamsorellana.org/page/2/
Let’s explore the object “uspPrintError”, which is stored on page 257:
DBCC traceon(3604)
DBCC page (adventureworks2008r2, 1, 257, 3)
DBCC traceoff(3604)
So, in the middle of that huge output, we can find the object on slot 13 (I will export just a part):
Slot 13 Offset 0x1a6b Length 765
Record Type = PRIMARY_RECORD Record Attributes = NULL_BITMAP VARIABLE_COLUMNS
Record Size = 765
Memory Dump @0x0000000009ABBA6B
0000000000000000: 30001100 0102797f 4d010000 00000000 †0…..y.M…….
0000000000000010: 000600c0 02002000 fd023801 02000000 †…À.. .ý.8…..
0000000000000020: 0d0a0d0a 2d2d2075 73705072 696e7445 †….– uspPrintE
0000000000000030: 72726f72 20707269 6e747320 6572726f †rror prints erro
0000000000000040: 7220696e 666f726d 6174696f 6e206162 †r information ab
0000000000000050: 6f757420 74686520 6572726f 72207468 †out the error th
0000000000000060: 61742063 61757365 64200d0a 2d2d2065 †at caused ..– e
0000000000000070: 78656375 74696f6e 20746f20 6a756d70 †xecution to jump
0000000000000080: 20746f20 74686520 43415443 4820626c † to the CATCH bl
0000000000000090: 6f636b20 6f662061 20545259 2e2e2e43 †ock of a TRY…C
00000000000000A0: 41544348 20636f6e 73747275 63742e20 †ATCH construct.
00000000000000B0: 0d0a2d2d 2053686f 756c6420 62652065 †..– Should be e
00000000000000C0: 78656375 74656420 66726f6d 20776974 †xecuted from wit
00000000000000D0: 68696e20 74686520 73636f70 65206f66 †hin the scope of
00000000000000E0: 20612043 41544348 20626c6f 636b206f † a CATCH block o
00000000000000F0: 74686572 77697365 200d0a2d 2d206974 †therwise ..– it
0000000000000100: 2077696c 6c207265 7475726e 20776974 † will return wit
0000000000000110: 686f7574 20707269 6e74696e 6720616e †hout printing an
0000000000000120: 79206572 726f7220 696e666f 726d6174 †y error informat
0000000000000130: 696f6e2e 0d0a4352 45415445 2050524f †ion…CREATE PRO
0000000000000140: 43454455 5245205b 64626f5d 2e5b7573 †CEDURE [dbo].[us
0000000000000150: 70507269 6e744572 726f725d 200d0a41 †pPrintError] ..A
So now, what if we…….
DROP PROCEDURE uspprinterror
… and quickly read the page content header:
DBCC traceon(3604)
DBCC page (adventureworks2008r2, 1, 257, 3)
DBCC traceoff(3604)
We will have the following output:
PAGE HEADER:
Page @0x0000000082582000
m_pageId = (1:257) m_headerVersion = 1 m_type = 1
m_typeFlagBits = 0x4 m_level = 0 m_flagBits = 0x0
m_objId (AllocUnitId.idObj) = 60 m_indexId (AllocUnitId.idInd) = 1 Metadata: AllocUnitId = 281474980642816
Metadata: PartitionId = 281474980642816 Metadata: IndexId = 1
Metadata: ObjectId = 60 m_prevPage = (1:23236) m_nextPage = (1:22959)
pminlen = 17 m_slotCnt = 35 m_freeCnt = 2889
m_freeData = 7528 m_reservedCnt = 0 m_lsn = (554:35134:9)
m_xactReserved = 0 m_xdesId = (0:1586506) m_ghostRecCnt = 1
We found that there’s a Ghost record (m_ghostRecCnt = 1), and we the have the following info in slot 13:
Slot 13 Offset 0x1a6b Length 765
Record Type = GHOST_DATA_RECORD Record Attributes = NULL_BITMAP VARIABLE_COLUMNS
Record Size = 765
Memory Dump @0x0000000009ABBA6B
0000000000000000: 3c001100 0102797f 4d010000 00000000 †<…..y.M…….
0000000000000010: 000600c0 02002000 fd023801 02000000 †…À.. .ý.8…..
0000000000000020: 0d0a0d0a 2d2d2075 73705072 696e7445 †….– uspPrintE
0000000000000030: 72726f72 20707269 6e747320 6572726f †rror prints erro
0000000000000040: 7220696e 666f726d 6174696f 6e206162 †r information ab
0000000000000050: 6f757420 74686520 6572726f 72207468 †out the error th
0000000000000060: 61742063 61757365 64200d0a 2d2d2065 †at caused ..– e
0000000000000070: 78656375 74696f6e 20746f20 6a756d70 †xecution to jump
0000000000000080: 20746f20 74686520 43415443 4820626c † to the CATCH bl
0000000000000090: 6f636b20 6f662061 20545259 2e2e2e43 †ock of a TRY…C
00000000000000A0: 41544348 20636f6e 73747275 63742e20 †ATCH construct.
00000000000000B0: 0d0a2d2d 2053686f 756c6420 62652065 †..– Should be e
00000000000000C0: 78656375 74656420 66726f6d 20776974 †xecuted from wit
00000000000000D0: 68696e20 74686520 73636f70 65206f66 †hin the scope of
00000000000000E0: 20612043 41544348 20626c6f 636b206f † a CATCH block o
Let’s wait a minute and check again…
DBCC traceon(3604)
DBCC page (adventureworks2008r2, 1, 257, 3)
DBCC traceoff(3604)
Output:
PAGE HEADER:
Page @0x0000000082582000
m_pageId = (1:257) m_headerVersion = 1 m_type = 1
m_typeFlagBits = 0x4 m_level = 0 m_flagBits = 0x0
m_objId (AllocUnitId.idObj) = 60 m_indexId (AllocUnitId.idInd) = 1 Metadata: AllocUnitId = 281474980642816
Metadata: PartitionId = 281474980642816 Metadata: IndexId = 1
Metadata: ObjectId = 60 m_prevPage = (1:23236) m_nextPage = (1:22959)
pminlen = 17 m_slotCnt = 34 m_freeCnt = 3656
m_freeData = 7528 m_reservedCnt = 0 m_lsn = (554:35140:3)
m_xactReserved = 0 m_xdesId = (0:1586506) m_ghostRecCnt = 0
m_tornBits = -1445838435
And for the Slot 13:
Slot 13 Offset 0x330 Length 40
Record Type = PRIMARY_RECORD Record Attributes = NULL_BITMAP VARIABLE_COLUMNS
Record Size = 40
Memory Dump @0x0000000009ABA330
0000000000000000: 30001100 01aaa153 4e000000 00000000 †0….ª¡SN…….
0000000000000010: 00060000 02002000 28003801 02000000 †…… .(.8…..
0000000000000020: 2828302e 30302929 †††††††††††††††††††((0.00))
The record m_ghostRecCnt is now 0, and we cannot find the procedure code anymore. Also the objid record is pointing to another item.
Anyway, if you run DBCC PAGE in option 2, you will still be able to find some object track!
Basically, the pages are “free” now, but the bytes stay untouched until something is written into that space. So, with luck, you can recover the object in an emergency situation. Awesome! :)
Friends, I hope you like this article and use it as a base for further learning because this is just a small part of how SQL Server works internally, and a DBA should be learning every single day.
If you have any question, suggestion, or other topic you want to talk about, feel free to contact me!
Share this
- Technical Track (969)
- Oracle (400)
- MySQL (137)
- Cloud (131)
- Open Source (90)
- Google Cloud (83)
- DBA Lounge (76)
- Microsoft SQL Server (76)
- Technical Blog (74)
- Big Data (52)
- AWS (49)
- Google Cloud Platform (47)
- Cassandra (44)
- DevOps (41)
- Azure (38)
- Pythian (33)
- Linux (30)
- Database (26)
- Podcasts (25)
- Site Reliability Engineering (25)
- Performance (24)
- SQL Server (24)
- Microsoft Azure (23)
- Oracle E-Business Suite (23)
- PostgreSQL (23)
- Oracle Database (22)
- Docker (21)
- Group Blog Posts (20)
- Security (20)
- DBA (19)
- Log Buffer (19)
- SQL (19)
- Exadata (18)
- Mongodb (18)
- Oracle Cloud Infrastructure (OCI) (18)
- Oracle Exadata (18)
- Automation (17)
- Hadoop (16)
- Oracleebs (16)
- Amazon RDS (15)
- Ansible (15)
- Ebs (15)
- Snowflake (15)
- ASM (13)
- BigQuery (13)
- Patching (13)
- RDS (13)
- Replication (13)
- Data (12)
- GenAI (12)
- Kubernetes (12)
- Oracle 12C (12)
- Advanced Analytics (11)
- Backup (11)
- LLM (11)
- Machine Learning (11)
- OCI (11)
- Rman (11)
- Cloud Migration (10)
- Datascape Podcast (10)
- Monitoring (10)
- R12 (10)
- 12C (9)
- AI (9)
- Apache Cassandra (9)
- Data Guard (9)
- Infrastructure (9)
- Oracle 19C (9)
- Oracle Applications (9)
- Python (9)
- Series (9)
- AWR (8)
- Amazon Web Services (AWS) (8)
- Articles (8)
- High Availability (8)
- Oracle EBS (8)
- Percona (8)
- Powershell (8)
- Recovery (8)
- Weblogic (8)
- Apache Beam (7)
- Backups (7)
- Data Governance (7)
- Goldengate (7)
- Innodb (7)
- Migration (7)
- Myrocks (7)
- OEM (7)
- Oracle Enterprise Manager (OEM) (7)
- Performance Tuning (7)
- Authentication (6)
- ChatGPT-4 (6)
- Data Enablement (6)
- Database Performance (6)
- E-Business Suite (6)
- Fmw (6)
- Grafana (6)
- Oracle Enterprise Manager (6)
- Orchestrator (6)
- Postgres (6)
- Rac (6)
- Renew Refresh Republish (6)
- RocksDB (6)
- Serverless (6)
- Upgrade (6)
- 19C (5)
- Azure Data Factory (5)
- Azure Synapse Analytics (5)
- Cpu (5)
- Data Visualization (5)
- Disaster Recovery (5)
- Error (5)
- Generative AI (5)
- Google BigQuery (5)
- Indexes (5)
- Love Letters To Data (5)
- Mariadb (5)
- Microsoft (5)
- Proxysql (5)
- Scala (5)
- Sql Server Administration (5)
- VMware (5)
- Windows (5)
- Xtrabackup (5)
- Airflow (4)
- Analytics (4)
- Apex (4)
- Best Practices (4)
- Centrally Managed Users (4)
- Cli (4)
- Cloud FinOps (4)
- Cloud Spanner (4)
- Cockroachdb (4)
- Configuration Management (4)
- Container (4)
- Data Management (4)
- Data Pipeline (4)
- Data Security (4)
- Data Strategy (4)
- Database Administrator (4)
- Database Management (4)
- Database Migration (4)
- Dataflow (4)
- Dbsat (4)
- Elasticsearch (4)
- Fahd Mirza (4)
- Fusion Middleware (4)
- Google (4)
- Io (4)
- Java (4)
- Kafka (4)
- Middleware (4)
- Mysql 8 (4)
- Network (4)
- Ocidtab (4)
- Opatch (4)
- Oracle Autonomous Database (Adb) (4)
- Oracle Cloud (4)
- Pitr (4)
- Post-Mortem Analysis (4)
- Prometheus (4)
- Redhat (4)
- September 9Th 2015 (4)
- Sql2016 (4)
- Ssl (4)
- Terraform (4)
- Workflow (4)
- 2Fa (3)
- Alwayson (3)
- Amazon Relational Database Service (Rds) (3)
- Apache Kafka (3)
- Apexexport (3)
- Aurora (3)
- Azure Sql Db (3)
- Cdb (3)
- ChatGPT (3)
- Cloud Armor (3)
- Cloud Database (3)
- Cloud Security (3)
- Cluster (3)
- Consul (3)
- Cosmos Db (3)
- Cost Management (3)
- Covid19 (3)
- Crontab (3)
- Data Analytics (3)
- Data Integration (3)
- Database 12C (3)
- Database Monitoring (3)
- Database Troubleshooting (3)
- Database Upgrade (3)
- Databases (3)
- Dataops (3)
- Dbt (3)
- Digital Transformation (3)
- ERP (3)
- Google Chrome (3)
- Google Cloud Sql (3)
- Graphite (3)
- Haproxy (3)
- Heterogeneous Database Migration (3)
- Hugepages (3)
- Inside Pythian (3)
- Installation (3)
- Json (3)
- Keras (3)
- Ldap (3)
- Liquibase (3)
- Love Letter (3)
- Lua (3)
- Mfa (3)
- Multitenant (3)
- Mysql 5.7 (3)
- Mysql Configuration (3)
- Nginx (3)
- Nodetool (3)
- Non-Tech Articles (3)
- Oem 13C (3)
- Oms (3)
- Oracle 18C (3)
- Oracle Data Guard (3)
- Oracle Live Sql (3)
- Oracle Rac (3)
- Patch (3)
- Perl (3)
- Pmm (3)
- Pt-Online-Schema-Change (3)
- Rdbms (3)
- Recommended (3)
- Remote Teams (3)
- Reporting (3)
- Reverse Proxy (3)
- S3 (3)
- Spark (3)
- Sql On The Edge (3)
- Sql Server Configuration (3)
- Sql Server On Linux (3)
- Ssis (3)
- Ssis Catalog (3)
- Stefan Knecht (3)
- Striim (3)
- Sysadmin (3)
- System Versioned (3)
- Systemd (3)
- Temporal Tables (3)
- Tensorflow (3)
- Tools (3)
- Tuning (3)
- Vasu Balla (3)
- Vault (3)
- Vulnerability (3)
- Waf (3)
- 18C (2)
- Adf (2)
- Adop (2)
- Agent (2)
- Agile (2)
- Amazon Data Migration Service (2)
- Amazon Ec2 (2)
- Amazon S3 (2)
- Apache Flink (2)
- Apple (2)
- Apps (2)
- Ashdump (2)
- Atp (2)
- Audit (2)
- Automatic Backups (2)
- Autonomous (2)
- Autoupgrade (2)
- Awr Data Mining (2)
- Azure Sql (2)
- Azure Sql Data Sync (2)
- Bash (2)
- Business (2)
- Business Intelligence (2)
- Caching (2)
- Cassandra Nodetool (2)
- Cdap (2)
- Certification (2)
- Cloning (2)
- Cloud Cost Optimization (2)
- Cloud Data Fusion (2)
- Cloud Hosting (2)
- Cloud Infrastructure (2)
- Cloud Shell (2)
- Cloud Sql (2)
- Cloudscape (2)
- Cluster Level Consistency (2)
- Conferences (2)
- Consul-Template (2)
- Containerization (2)
- Containers (2)
- Cosmosdb (2)
- Costs (2)
- Cql (2)
- Cqlsh (2)
- Cyber Security (2)
- Data Discovery (2)
- Data Migration (2)
- Data Quality (2)
- Data Streaming (2)
- Data Warehouse (2)
- Database Consulting (2)
- Database Migrations (2)
- Dataguard (2)
- Datapump (2)
- Ddl (2)
- Debezium (2)
- Dictionary Views (2)
- Dms (2)
- Docker-Composer (2)
- Dr (2)
- Duplicate (2)
- Ecc (2)
- Elastic (2)
- Elastic Stack (2)
- Em12C (2)
- Encryption (2)
- Enterprise Data Platform (EDP) (2)
- Enterprise Manager (2)
- Etl (2)
- Events (2)
- Exachk (2)
- Filter Driver (2)
- Flume (2)
- Full Text Search (2)
- Galera (2)
- Gemini (2)
- General Purpose Ssd (2)
- Gh-Ost (2)
- Gke (2)
- Google Workspace (2)
- Hanganalyze (2)
- Hdfs (2)
- Health Check (2)
- Historical Trends (2)
- Incremental (2)
- Infiniband (2)
- Infrastructure As Code (2)
- Innodb Cluster (2)
- Innodb File Structure (2)
- Innodb Group Replication (2)
- Install (2)
- Internals (2)
- Java Web Start (2)
- Kibana (2)
- Log (2)
- Log4J (2)
- Logs (2)
- Memory (2)
- Merge Replication (2)
- Metrics (2)
- Mutex (2)
- MySQLShell (2)
- NLP (2)
- Neo4J (2)
- Node.Js (2)
- Nosql (2)
- November 11Th 2015 (2)
- Ntp (2)
- Oci Iam (2)
- Oem12C (2)
- Omspatcher (2)
- Opatchauto (2)
- Open Source Database (2)
- Operational Excellence (2)
- Oracle 11G (2)
- Oracle Datase (2)
- Oracle Extended Manager (Oem) (2)
- Oracle Flashback (2)
- Oracle Forms (2)
- Oracle Installation (2)
- Oracle Io Testing (2)
- Pdb (2)
- Podcast (2)
- Puppet (2)
- Pythian Europe (2)
- R12.2 (2)
- Redshift (2)
- Remote DBA (2)
- Remote Sre (2)
- SAP (2)
- SAP HANA Cloud (2)
- Sap Migration (2)
- Scale (2)
- Schema (2)
- September 30Th 2015 (2)
- September 3Rd 2015 (2)
- Shell (2)
- Simon Pane (2)
- Single Sign-On (2)
- Sql Server On Gke (2)
- Sqlplus (2)
- Sre (2)
- Ssis Catalog Error (2)
- Ssisdb (2)
- Standby (2)
- Statspack Mining (2)
- Systemstate Dump (2)
- Tablespace (2)
- Technical Training (2)
- Tempdb (2)
- Tfa (2)
- Throughput (2)
- Tls (2)
- Tombstones (2)
- Transactional Replication (2)
- User Groups (2)
- Vagrant (2)
- Variables (2)
- Virtual Machine (2)
- Virtual Machines (2)
- Virtualbox (2)
- Web Application Firewall (2)
- Webinars (2)
- X5 (2)
- scalability (2)
- //Build2019 (1)
- 11G (1)
- 12.1 (1)
- 12Cr1 (1)
- 12Cr2 (1)
- 18C Grid Installation (1)
- 2022 (1)
- 2022 Snowflake Summit (1)
- AI Platform (1)
- AI Summit (1)
- Actifio (1)
- Active Directory (1)
- Adaptive Hash Index (1)
- Adf Custom Email (1)
- Adobe Flash (1)
- Adrci (1)
- Advanced Data Services (1)
- Afd (1)
- After Logon Trigger (1)
- Ahf (1)
- Aix (1)
- Akka (1)
- Alloydb (1)
- Alter Table (1)
- Always On (1)
- Always On Listener (1)
- Alwayson With Gke (1)
- Amazon (1)
- Amazon Athena (1)
- Amazon Aurora Backtrack (1)
- Amazon Efs (1)
- Amazon Redshift (1)
- Amazon Sagemaker (1)
- Amazon Vpc Flow Logs (1)
- Amdu (1)
- Analysis (1)
- Analytical Models (1)
- Analyzing Bigquery Via Sheets (1)
- Anisble (1)
- Annual Mysql Community Dinner (1)
- Anthos (1)
- Apache (1)
- Apache Nifi (1)
- Apache Spark (1)
- Application Migration (1)
- Architect (1)
- Architecture (1)
- Ash (1)
- Asmlib (1)
- Atlas CLI (1)
- Audit In Postgres (1)
- Audit In Postgresql (1)
- Auto Failover (1)
- Auto Increment (1)
- Auto Index (1)
- Autoconfig (1)
- Automated Reports (1)
- Automl (1)
- Autostart (1)
- Awr Mining (1)
- Aws Glue (1)
- Aws Lake Formation (1)
- Aws Lambda (1)
- Azure Analysis Services (1)
- Azure Blob Storage (1)
- Azure Cognitive Search (1)
- Azure Data (1)
- Azure Data Lake (1)
- Azure Data Lake Analytics (1)
- Azure Data Lake Store (1)
- Azure Data Migration Service (1)
- Azure Dma (1)
- Azure Dms (1)
- Azure Document Intelligence (1)
- Azure Integration Runtime (1)
- Azure OpenAI (1)
- Azure Sql Data Warehouse (1)
- Azure Sql Dw (1)
- Azure Sql Managed Instance (1)
- Azure Vm (1)
- Backup For Sql Server (1)
- Bacpac (1)
- Bag (1)
- Bare Metal Solution (1)
- Batch Operation (1)
- Batches In Cassandra (1)
- Beats (1)
- Best Practice (1)
- Bi Publisher (1)
- Binary Logging (1)
- Bind Variables (1)
- Bitnami (1)
- Blob Storage Endpoint (1)
- Blockchain (1)
- Browsers (1)
- Btp Architecture (1)
- Btp Components (1)
- Buffer Pool (1)
- Bug (1)
- Bugs (1)
- Build 2019 Updates (1)
- Build Cassandra (1)
- Bundle Patch (1)
- Bushy Join (1)
- Business Continuity (1)
- Business Insights (1)
- Business Process Modelling (1)
- Business Reputation (1)
- CAPEX (1)
- Capacity Planning (1)
- Career (1)
- Career Development (1)
- Cassandra-Cli (1)
- Catcon.Pm (1)
- Catctl.Pl (1)
- Catupgrd.Sql (1)
- Cbo (1)
- Cdb Duplication (1)
- Certificate (1)
- Certificate Management (1)
- Chaos Engineering (1)
- Cheatsheet (1)
- Checkactivefilesandexecutables (1)
- Chmod (1)
- Chown (1)
- Chrome Enterprise (1)
- Chrome Security (1)
- Cl-Series (1)
- Cleanup (1)
- Cloud Browser (1)
- Cloud Build (1)
- Cloud Consulting (1)
- Cloud Data Warehouse (1)
- Cloud Database Management (1)
- Cloud Dataproc (1)
- Cloud Foundry (1)
- Cloud Manager (1)
- Cloud Migations (1)
- Cloud Networking (1)
- Cloud SQL Replica (1)
- Cloud Scheduler (1)
- Cloud Services (1)
- Cloud Strategies (1)
- Cloudformation (1)
- Cluster Resource (1)
- Cmo (1)
- Cockroach Db (1)
- Coding Benchmarks (1)
- Colab (1)
- Collectd (1)
- Columnar (1)
- Communication Plans (1)
- Community (1)
- Compact Storage (1)
- Compaction (1)
- Compliance (1)
- Compression (1)
- Compute Instances (1)
- Compute Node (1)
- Concurrent Manager (1)
- Concurrent Processing (1)
- Configuration (1)
- Consistency Level (1)
- Consolidation (1)
- Conversational AI (1)
- Covid-19 (1)
- Cpu Patching (1)
- Cqlsstablewriter (1)
- Crash (1)
- Create Catalog Error (1)
- Create_File_Dest (1)
- Credentials (1)
- Cross Platform (1)
- CrowdStrike (1)
- Crsctl (1)
- Custom Instance Images (1)
- Cve-2022-21500 (1)
- Cvu (1)
- Cypher Queries (1)
- DBSAT 3 (1)
- Dacpac (1)
- Dag (1)
- Data Analysis (1)
- Data Analytics Platform (1)
- Data Box (1)
- Data Classification (1)
- Data Cleansing (1)
- Data Encryption (1)
- Data Engineering (1)
- Data Estate (1)
- Data Flow Management (1)
- Data Insights (1)
- Data Integrity (1)
- Data Lake (1)
- Data Leader (1)
- Data Lifecycle Management (1)
- Data Lineage (1)
- Data Masking (1)
- Data Mesh (1)
- Data Migration Assistant (1)
- Data Migration Service (1)
- Data Mining (1)
- Data Modeling (1)
- Data Monetization (1)
- Data Policy (1)
- Data Profiling (1)
- Data Protection (1)
- Data Retention (1)
- Data Safe (1)
- Data Sheets (1)
- Data Summit (1)
- Data Vault (1)
- Data Warehouse Modernization (1)
- Database Auditing (1)
- Database Consultant (1)
- Database Link (1)
- Database Modernization (1)
- Database Provisioning (1)
- Database Provisioning Failed (1)
- Database Replication (1)
- Database Scaling (1)
- Database Schemas (1)
- Database Security (1)
- Databricks (1)
- Datadog (1)
- Datafile (1)
- Datapatch (1)
- Dataprivacy (1)
- Datascape 59 (1)
- Datasets (1)
- Datastax Cassandra (1)
- Datastax Opscenter (1)
- Datasync Error (1)
- Db_Create_File_Dest (1)
- Dbaas (1)
- Dbatools (1)
- Dbcc Checkident (1)
- Dbms_Cloud (1)
- Dbms_File_Transfer (1)
- Dbms_Metadata (1)
- Dbms_Service (1)
- Dbms_Stats (1)
- Dbupgrade (1)
- Deep Learning (1)
- Delivery (1)
- Devd (1)
- Dgbroker (1)
- Dialogflow (1)
- Dict0Dict (1)
- Did You Know (1)
- Direct Path Read Temp (1)
- Disk Groups (1)
- Disk Management (1)
- Diskgroup (1)
- Dispatchers (1)
- Distributed Ag (1)
- Distribution Agent (1)
- Documentation (1)
- Download (1)
- Dp Agent (1)
- Duet AI (1)
- Duplication (1)
- Dynamic Sampling (1)
- Dynamic Tasks (1)
- E-Business Suite Cpu Patching (1)
- E-Business Suite Patching (1)
- Ebs Sso (1)
- Ec2 (1)
- Edb Postgresql Advanced Server (1)
- Edb Postgresql Password Verify Function (1)
- Editions (1)
- Edp (1)
- El Carro (1)
- Elassandra (1)
- Elk Stack (1)
- Em13Cr2 (1)
- Emcli (1)
- End of Life (1)
- Engineering (1)
- Enqueue (1)
- Enterprise (1)
- Enterprise Architecture (1)
- Enterprise Command Centers (1)
- Enterprise Manager Command Line Interface (Em Cli (1)
- Enterprise Plus (1)
- Episode 58 (1)
- Error Handling (1)
- Exacc (1)
- Exacheck (1)
- Exacs (1)
- Exadata Asr (1)
- Execution (1)
- Executive Sponsor (1)
- Expenditure (1)
- Export Sccm Collection To Csv (1)
- External Persistent Volumes (1)
- Fail (1)
- Failed Upgrade (1)
- Failover In Postgresql (1)
- Fall 2021 (1)
- Fast Recovery Area (1)
- FinOps Strategy (1)
- Flash Recovery Area (1)
- Flashback (1)
- Fnd (1)
- Fndsm (1)
- Force_Matching_Signature (1)
- Fra Full (1)
- Framework (1)
- Freebsd (1)
- Fsync (1)
- Function-Based Index (1)
- GCVE Architecture (1)
- GPQA (1)
- Gaming (1)
- Garbagecollect (1)
- Gcp Compute (1)
- Gcp-Spanner (1)
- Geography (1)
- Geth (1)
- Getmospatch (1)
- Git (1)
- Global Analytics (1)
- Gmail (1)
- Gmail Security (1)
- Google Analytics (1)
- Google Cloud Architecture Framework (1)
- Google Cloud Data Services (1)
- Google Cloud Partner (1)
- Google Cloud Spanner (1)
- Google Cloud VMware Engine (1)
- Google Compute Engine (1)
- Google Dataflow (1)
- Google Datalab (1)
- Google Grab And Go (1)
- Google Sheets (1)
- Gp2 (1)
- Graph Algorithms (1)
- Graph Databases (1)
- Graph Inferences (1)
- Graph Theory (1)
- GraphQL (1)
- Graphical User Interface (Gui) (1)
- Grid (1)
- Grid Infrastructure (1)
- Griddisk Resize (1)
- Grp (1)
- Guaranteed Restore Point (1)
- Guid Mismatch (1)
- HR Technology (1)
- HRM (1)
- Ha (1)
- Hang (1)
- Hashicorp (1)
- Hbase (1)
- Hcc (1)
- Hdinsight (1)
- Healthcheck (1)
- Hemantgiri S. Goswami (1)
- Hortonworks (1)
- How To Install Ssrs (1)
- Hr (1)
- Httpchk (1)
- Https (1)
- Huge Pages (1)
- HumanEval (1)
- Hung Database (1)
- Hybrid Columnar Compression (1)
- Hyper-V (1)
- Hyperscale (1)
- Hypothesis Driven Development (1)
- Ibm (1)
- Identity Management (1)
- Idm (1)
- Ilom (1)
- Imageinfo (1)
- Impdp (1)
- In Place Upgrade (1)
- Incident Response (1)
- Indempotent (1)
- Indexing In Mongodb (1)
- Influxdb (1)
- Information (1)
- Infrastructure As A Code (1)
- Injection (1)
- Innobackupex (1)
- Innodb Concurrency (1)
- Innodb Flush Method (1)
- Insights (1)
- Installing (1)
- Instance Cloning (1)
- Integration Services (1)
- Integrations (1)
- Interactive_Timeout (1)
- Interval Partitioning (1)
- Invisible Indexes (1)
- Io1 (1)
- IoT (1)
- Iops (1)
- Iphone (1)
- Ipv6 (1)
- Iscsi (1)
- Iscsi-Initiator-Utils (1)
- Iscsiadm (1)
- Issues (1)
- It Industry (1)
- It Teams (1)
- JMX Metrics (1)
- Jared Still (1)
- Javascript (1)
- Jdbc (1)
- Jinja2 (1)
- Jmx (1)
- Jmx Monitoring (1)
- Jvm (1)
- Jython (1)
- K8S (1)
- Kernel (1)
- Key Btp Components (1)
- Kfed (1)
- Kill Sessions (1)
- Knapsack (1)
- Kubeflow (1)
- LMSYS Chatbot Arena (1)
- Large Pages (1)
- Latency (1)
- Latest News (1)
- Leadership (1)
- Leap Second (1)
- Limits (1)
- Line 1 (1)
- Linkcolumn (1)
- Linux Host Monitoring (1)
- Linux Storage Appliance (1)
- Listener (1)
- Loadavg (1)
- Lock_Sga (1)
- Locks (1)
- Log File Switch (Archiving Needed) (1)
- Logfile (1)
- Looker (1)
- Lvm (1)
- MMLU (1)
- Managed Instance (1)
- Managed Services (1)
- Management (1)
- Management Servers (1)
- Marketing (1)
- Marketing Analytics (1)
- Martech (1)
- Masking (1)
- Megha Bedi (1)
- Metadata (1)
- Method-R Workbench (1)
- Metric (1)
- Metric Extensions (1)
- Michelle Gutzait (1)
- Microservices (1)
- Microsoft Azure Sql Database (1)
- Microsoft Build (1)
- Microsoft Build 2019 (1)
- Microsoft Ignite (1)
- Microsoft Inspire 2019 (1)
- Migrate (1)
- Migrating Ssis Catalog (1)
- Migrating To Azure Sql (1)
- Migration Checklist (1)
- Mirroring (1)
- Mismatch (1)
- Model Governance (1)
- Monetization (1)
- MongoDB Atlas (1)
- MongoDB Compass (1)
- Ms Excel (1)
- Msdtc (1)
- Msdtc In Always On (1)
- Msdtc In Cluster (1)
- Multi-IP (1)
- Multicast (1)
- Multipath (1)
- My.Cnf (1)
- MySQL Shell Logical Backup (1)
- MySQLDump (1)
- Mysql Enterprise (1)
- Mysql Plugin For Oracle Enterprise Manager (1)
- Mysql Replication Filters (1)
- Mysql Server (1)
- Mysql-Python (1)
- Nagios (1)
- Ndb (1)
- Net_Read_Timeout (1)
- Net_Write_Timeout (1)
- Netcat (1)
- Newsroom (1)
- Nfs (1)
- Nifi (1)
- Node (1)
- November 10Th 2015 (1)
- November 6Th 2015 (1)
- Null Columns (1)
- Nullipotent (1)
- OPEX (1)
- ORAPKI (1)
- O_Direct (1)
- Oacore (1)
- October 21St 2015 (1)
- October 6Th 2015 (1)
- October 8Th 2015 (1)
- Oda (1)
- Odbcs (1)
- Odbs (1)
- Odi (1)
- Oel (1)
- Ohs (1)
- Olvm (1)
- On-Prem To Azure Sql (1)
- On-Premises (1)
- Onclick (1)
- Open.Canada.Ca (1)
- Openstack (1)
- Operating System Monitoring (1)
- Oplog (1)
- Opsworks (1)
- Optimization (1)
- Optimizer (1)
- Ora-01852 (1)
- Ora-7445 (1)
- Oracle 19 (1)
- Oracle 20C (1)
- Oracle Cursor (1)
- Oracle Database 12.2 (1)
- Oracle Database Appliance (1)
- Oracle Database Se2 (1)
- Oracle Database Standard Edition 2 (1)
- Oracle Database Upgrade (1)
- Oracle Database@Google Cloud (1)
- Oracle Exadata Smart Scan (1)
- Oracle Licensing (1)
- Oracle Linux Virtualization Manager (1)
- Oracle Oda (1)
- Oracle Openworld (1)
- Oracle Parallelism (1)
- Oracle Rdbms (1)
- Oracle Real Application Clusters (1)
- Oracle Reports (1)
- Oracle Security (1)
- Oracle Wallet (1)
- Orasrp (1)
- Organizational Change (1)
- Orion (1)
- Os (1)
- Osbws_Install.Jar (1)
- Oui Gui (1)
- Output (1)
- Owox (1)
- Paas (1)
- Package Deployment Wizard Error (1)
- Parallel Execution (1)
- Parallel Query (1)
- Parallel Query Downgrade (1)
- Partitioning (1)
- Partitions (1)
- Password (1)
- Password Change (1)
- Password Recovery (1)
- Password Verify Function In Postgresql (1)
- Patches (1)
- Patchmgr (1)
- Pdb Duplication (1)
- Penalty (1)
- Perfomrance (1)
- Performance Schema (1)
- Pg 15 (1)
- Pg_Rewind (1)
- Pga (1)
- Pipeline Debugging (1)
- Pivot (1)
- Planning (1)
- Plsql (1)
- Policy (1)
- Polybase (1)
- Post-Acquisition (1)
- Post-Covid It (1)
- Postgresql Complex Password (1)
- Postgresql With Repmgr Integration (1)
- Power Bi (1)
- Pq (1)
- Preliminar Connection (1)
- Preliminary Connection (1)
- Privatecloud (1)
- Process Mining (1)
- Production (1)
- Productivity (1)
- Profile In Edb Postgresql (1)
- Programming (1)
- Prompt Engineering (1)
- Provisioned Iops (1)
- Provisiones Iops (1)
- Proxy Monitoring (1)
- Psu (1)
- Public Cloud (1)
- Pubsub (1)
- Purge (1)
- Purge Thread (1)
- Pythian Blackbird Acquisition (1)
- Pythian Goodies (1)
- Pythian News (1)
- Python Pandas (1)
- Query Performance (1)
- Quicksight (1)
- Quota Limits (1)
- R12 R12.2 Cp Concurrent Processing Abort (1)
- R12.1.3 (1)
- REF! (1)
- Ram Cache (1)
- Rbac (1)
- Rdb (1)
- Rds_File_Util (1)
- Read Free Replication (1)
- Read Latency (1)
- Read Only (1)
- Read Replica (1)
- Reboot (1)
- Recruiting (1)
- Redo Size (1)
- Relational Database Management System (1)
- Release (1)
- Release Automation (1)
- Repair (1)
- Replication Compatibility (1)
- Replication Error (1)
- Repmgr (1)
- Repmgrd (1)
- Reporting Services 2019 (1)
- Resiliency Planning (1)
- Resource Manager (1)
- Resources (1)
- Restore (1)
- Restore Point (1)
- Retail (1)
- Rhel (1)
- Risk (1)
- Risk Management (1)
- Rocksrb (1)
- Role In Postgresql (1)
- Rollback (1)
- Rolling Patch (1)
- Row0Purge (1)
- Rpm (1)
- Rule "Existing Clustered Or Clustered-Prepared In (1)
- Running Discovery On Remote Machine (1)
- SQL Optimization (1)
- SQL Tracing (1)
- SSRS Administration (1)
- SaaS (1)
- Sap Assessment (1)
- Sap Assessment Report (1)
- Sap Backup Restore (1)
- Sap Btp Architecture (1)
- Sap Btp Benefits (1)
- Sap Btp Model (1)
- Sap Btp Services (1)
- Sap Homogenous System Copy Method (1)
- Sap Landscape Copy (1)
- Sap Migration Assessment (1)
- Sap On Mssql (1)
- Sap System Copy (1)
- Sar (1)
- Scaling Ir (1)
- Sccm (1)
- Sccm Powershell (1)
- Scheduler (1)
- Scheduler_Job (1)
- Schedulers (1)
- Scheduling (1)
- Scott Mccormick (1)
- Scripts (1)
- Sdp (1)
- Secrets (1)
- Securing Sql Server (1)
- Security Compliance (1)
- Sed (Stream Editor) (1)
- Self Hosted Ir (1)
- Semaphore (1)
- Seps (1)
- September 11Th 2015 (1)
- Serverless Computing (1)
- Serverless Framework (1)
- Service Broker (1)
- Service Bus (1)
- Shared Connections (1)
- Shared Storage (1)
- Shellshock (1)
- Signals (1)
- Silent (1)
- Slave (1)
- Slob (1)
- Smart Scan (1)
- Smtp (1)
- Snapshot (1)
- Snowday Fall 2021 (1)
- Socat (1)
- Software Development (1)
- Software Engineering (1)
- Solutions Architecture (1)
- Spanner-Backups (1)
- Sphinx (1)
- Split Brain In Postgresql (1)
- Spm (1)
- Sql Agent (1)
- Sql Backup To Url Error (1)
- Sql Cluster Installer Hang (1)
- Sql Database (1)
- Sql Developer (1)
- Sql On Linux (1)
- Sql Server 2014 (1)
- Sql Server 2016 (1)
- Sql Server Agent On Linux (1)
- Sql Server Backups (1)
- Sql Server Denali Is Required To Install Integrat (1)
- Sql Server Health Check (1)
- Sql Server Troubleshooting On Linux (1)
- Sql Server Version (1)
- Sql Setup (1)
- Sql Vm (1)
- Sql2K19Ongke (1)
- Sqldatabase Serverless (1)
- Ssh User Equivalence (1)
- Ssis Denali Error (1)
- Ssis Install Error E Xisting Clustered Or Cluster (1)
- Ssis Package Deployment Error (1)
- Ssisdb Master Key (1)
- Ssisdb Restore Error (1)
- Sso (1)
- Ssrs 2019 (1)
- Sstable2Json (1)
- Sstableloader (1)
- Sstablesimpleunsortedwriter (1)
- Stack Dump (1)
- Standard Edition (1)
- Startup Process (1)
- Statistics (1)
- Statspack (1)
- Statspack Data Mining (1)
- Statspack Erroneously Reporting (1)
- Statspack Issues (1)
- Storage (1)
- Stored Procedure (1)
- Strategies (1)
- Streaming (1)
- Sunos (1)
- Swap (1)
- Swapping (1)
- Switch (1)
- Syft (1)
- Synapse (1)
- Sync Failed There Is Not Enough Space On The Disk (1)
- Sys Schema (1)
- System Function (1)
- Systems Administration (1)
- T-Sql (1)
- Table Optimization (1)
- Tablespace Growth (1)
- Tablespaces (1)
- Tags (1)
- Tar (1)
- Tde (1)
- Team Management (1)
- Tech Debt (1)
- Technology (1)
- Telegraf (1)
- Tempdb Encryption (1)
- Templates (1)
- Temporary Tablespace (1)
- Tenserflow (1)
- Teradata (1)
- Testing New Cassandra Builds (1)
- There Is Not Enough Space On The Disk (1)
- Thick Data (1)
- Third-Party Data (1)
- Thrift (1)
- Thrift Data (1)
- Tidb (1)
- Time Series (1)
- Time-Drift (1)
- Tkprof (1)
- Tmux (1)
- Tns (1)
- Trace (1)
- Tracefile (1)
- Training (1)
- Transaction Log (1)
- Transactions (1)
- Transformation Navigator (1)
- Transparent Data Encryption (1)
- Trigger (1)
- Triggers On Memory-Optimized Tables Must Use With (1)
- Troubleshooting (1)
- Tungsten (1)
- Tvdxtat (1)
- Twitter (1)
- U-Sql (1)
- UNDO Tablespace (1)
- Upgrade Issues (1)
- Uptime (1)
- Uptrade (1)
- Url Backup Error (1)
- Usability (1)
- Use Cases (1)
- User (1)
- User Defined Compactions (1)
- Utilization (1)
- Utl_Smtp (1)
- VDI Jump Host (1)
- Validate Structure (1)
- Validate_Credentials (1)
- Value (1)
- Velocity (1)
- Vertex AI (1)
- Vertica (1)
- Vertical Slicing (1)
- Videos (1)
- Virtual Private Cloud (1)
- Virtualization (1)
- Vision (1)
- Vpn (1)
- Wait_Timeout (1)
- Wallet (1)
- Webhook (1)
- Weblogic Connection Filters (1)
- Webscale Database (1)
- Windows 10 (1)
- Windows Powershell (1)
- WiredTiger (1)
- With Native_Compilation (1)
- Word (1)
- Workshop (1)
- Workspace Security (1)
- Xbstream (1)
- Xml Publisher (1)
- Zabbix (1)
- dbms_Monitor (1)
- postgresql 16 (1)
- sqltrace (1)
- tracing (1)
- vSphere (1)
- xml (1)
- October 2024 (2)
- September 2024 (7)
- August 2024 (4)
- July 2024 (2)
- June 2024 (6)
- May 2024 (3)
- April 2024 (2)
- February 2024 (2)
- January 2024 (11)
- December 2023 (10)
- November 2023 (11)
- October 2023 (10)
- September 2023 (8)
- August 2023 (7)
- July 2023 (2)
- June 2023 (13)
- May 2023 (4)
- April 2023 (6)
- March 2023 (10)
- February 2023 (6)
- January 2023 (5)
- December 2022 (10)
- November 2022 (10)
- October 2022 (10)
- September 2022 (13)
- August 2022 (16)
- July 2022 (12)
- June 2022 (13)
- May 2022 (11)
- April 2022 (4)
- March 2022 (5)
- February 2022 (4)
- January 2022 (14)
- December 2021 (16)
- November 2021 (11)
- October 2021 (7)
- September 2021 (11)
- August 2021 (6)
- July 2021 (9)
- June 2021 (4)
- May 2021 (8)
- April 2021 (16)
- March 2021 (16)
- February 2021 (6)
- January 2021 (12)
- December 2020 (12)
- November 2020 (17)
- October 2020 (11)
- September 2020 (10)
- August 2020 (11)
- July 2020 (13)
- June 2020 (6)
- May 2020 (9)
- April 2020 (18)
- March 2020 (21)
- February 2020 (13)
- January 2020 (15)
- December 2019 (10)
- November 2019 (11)
- October 2019 (12)
- September 2019 (16)
- August 2019 (15)
- July 2019 (10)
- June 2019 (16)
- May 2019 (20)
- April 2019 (21)
- March 2019 (14)
- February 2019 (18)
- January 2019 (18)
- December 2018 (5)
- November 2018 (16)
- October 2018 (12)
- September 2018 (20)
- August 2018 (27)
- July 2018 (31)
- June 2018 (34)
- May 2018 (28)
- April 2018 (27)
- March 2018 (17)
- February 2018 (8)
- January 2018 (20)
- December 2017 (14)
- November 2017 (4)
- October 2017 (1)
- September 2017 (3)
- August 2017 (5)
- July 2017 (4)
- June 2017 (2)
- May 2017 (7)
- April 2017 (7)
- March 2017 (8)
- February 2017 (8)
- January 2017 (5)
- December 2016 (3)
- November 2016 (4)
- October 2016 (8)
- September 2016 (9)
- August 2016 (10)
- July 2016 (9)
- June 2016 (8)
- May 2016 (13)
- April 2016 (16)
- March 2016 (13)
- February 2016 (11)
- January 2016 (6)
- December 2015 (11)
- November 2015 (11)
- October 2015 (5)
- September 2015 (16)
- August 2015 (4)
- July 2015 (1)
- June 2015 (3)
- May 2015 (6)
- April 2015 (5)
- March 2015 (5)
- February 2015 (4)
- January 2015 (3)
- December 2014 (7)
- October 2014 (4)
- September 2014 (6)
- August 2014 (6)
- July 2014 (16)
- June 2014 (7)
- May 2014 (6)
- April 2014 (5)
- March 2014 (4)
- February 2014 (10)
- January 2014 (6)
- December 2013 (8)
- November 2013 (12)
- October 2013 (9)
- September 2013 (6)
- August 2013 (7)
- July 2013 (9)
- June 2013 (7)
- May 2013 (7)
- April 2013 (4)
- March 2013 (7)
- February 2013 (4)
- January 2013 (4)
- December 2012 (6)
- November 2012 (8)
- October 2012 (9)
- September 2012 (3)
- August 2012 (5)
- July 2012 (5)
- June 2012 (7)
- May 2012 (11)
- April 2012 (1)
- March 2012 (8)
- February 2012 (1)
- January 2012 (6)
- December 2011 (8)
- November 2011 (5)
- October 2011 (9)
- September 2011 (6)
- August 2011 (4)
- July 2011 (1)
- June 2011 (1)
- May 2011 (5)
- April 2011 (2)
- February 2011 (2)
- January 2011 (2)
- December 2010 (1)
- November 2010 (7)
- October 2010 (3)
- September 2010 (8)
- August 2010 (2)
- July 2010 (4)
- June 2010 (7)
- May 2010 (2)
- April 2010 (1)
- March 2010 (3)
- February 2010 (3)
- January 2010 (2)
- November 2009 (6)
- October 2009 (6)
- August 2009 (3)
- July 2009 (3)
- June 2009 (3)
- May 2009 (2)
- April 2009 (8)
- March 2009 (6)
- February 2009 (4)
- January 2009 (3)
- November 2008 (3)
- October 2008 (7)
- September 2008 (6)
- August 2008 (9)
- July 2008 (9)
- June 2008 (9)
- May 2008 (9)
- April 2008 (8)
- March 2008 (4)
- February 2008 (3)
- January 2008 (3)
- December 2007 (2)
- November 2007 (7)
- October 2007 (1)
- August 2007 (4)
- July 2007 (3)
- June 2007 (8)
- May 2007 (4)
- April 2007 (2)
- March 2007 (2)
- February 2007 (5)
- January 2007 (8)
- December 2006 (1)
- November 2006 (3)
- October 2006 (4)
- September 2006 (3)
- July 2006 (1)
- May 2006 (2)
- April 2006 (1)
- July 2005 (1)
No Comments Yet
Let us know what you think